:030000000233BE0A
:0C33BE0078FFE4F6D8FD75815802340554
:100F4E0020000A3C2E2E2E3E004950436F6E6E65D9
:100F5E0063745245510A004950436F6E6E65637457
:100F6E00000A49504E6F41434B210A003E432C5616
:100F7E002C43432CC0E4E0EFF2E5F020D1E8EDEA9B
:100F8E00EEEC49500A003E432C4D41432C253032A5
:100F9E0062583A25303262583A25303262583A2534
:100FAE00303262583A25303262583A253032625821
:100FBE002C4D414320E0E4F0E5F10A003E432C566F
:100FCE0045522C20332E3220EEF22025732025732D
:100FDE002CC2E5F0F1E8FF20495020ECEEE4F3EBF3
:100FEE00FF0A004F63742030382032303134003124
:100FFE00353A34393A3130003E432C4C442C505261
:10100E004F473A2020202020202020202020202062
:10101E0020202020202020202020202020202020C2
:10102E0020202020202020202020202020202020B2
:10103E0020202020202020202020202020202020A2
:10104E0020202020202020202CC4E0F2E020EFF0F1
:10105E00EEF8E8E2EAE828F4E0E9EB290A003E2A95
:10106E002C312CCEF1EDEEE2EDFBE520EFE0F0E0E1
:10107E00ECE5F2F0FB20F1E5F2E5E2EEE3EE20E83E
:10108E00EDF2E5F0F4E5E9F1E00A003E412C4130E5
:10109E00312C2562752E2562752E2562752E2562E0
:1010AE00752C495020E0E4F0E5F120E0E4E0EFF2A9
:1010BE00E5F0E00A003E412C4130342C2562752EBD
:1010CE002562752E2562752E2562752CCCE0F1EA0F
:1010DE00E020F1E5F2E80A003E412C4130352C25A6
:1010EE0062752E2562752E2562752E2562752CD899
:1010FE00EBFEE70A003E2A2C312CCFE0F0E0ECE5C7
:10110E00F2F0FB20EEE1ECE5EDE020EFEE20EFF06B
:10111E00EEF2EEEAEEEBF3205544503937320A0088
:10112E003E412C4130322C2562752E2562752E25BE
:10113E0062752E2562752C495020E0E4F0E5F12011
:10114E00EEF1ED2E20F1E5F0E2E5F0E00A003E4191
:10115E002C4130332C2562752E2562752E25627535
:10116E002E2562752C495020E0E4F0E5F120F0E5E3
:10117E00E72E20F1E5F0E2E5F0E00A003E422C53C6
:10118E0030322C2562752CCEE1ECE5ED20F120F10C
:10119E00E5F0E2E5F0EEEC20E1E5E720EAE2E8F248
:1011AE00E0EDF6E8E90A003E422C5330332C25627E
:1011BE00752CCFE5F0E5E7E0EFF3F1EA20EFF0E88C
:1011CE0020EFEEF2E5F0E520F1E2FFE7E820F12076
:1011DE00F1E5F0E2E5F0EEEC0A003E422C53303839
:1011EE002C2562752CCCE5E4EBE5EDEDFBE9204911
:1011FE005020EAE0EDE0EB28E7E0E4E5F0E6EAE097
:10120E0020E4EE203520F1E5EA290A003E454E4461
:10121E000A000A44756D705820202020203030209E
:10122E0030312030322030332030342030352030F1
:10123E0036203037203038203039203041203042AF
:10124E00203043203044203045203046000A3A00FA
:10125E003A20000A000A44756D7044202020202098
:10126E0030302030312030322030332030342030B6
:10127E00352030362030372030382030392030417C
:10128E00203042203043203044203045203046006C
:10129E00457272206B657900526420656570726FBD
:1012AE006D0A005264204D454D0A00526420436F72
:1012BE0064650A00577269746520436F64650A009D
:1012CE0044656275674950204F4E0A004465627549
:1012DE00674950204F46460A00446562756755734C
:1012EE006572204F6E0A00446562756755736572AC
:1012FE00204F46460A0044656275674D7367204F5E
:10130E006E0A0044656275674D7367204F46460A44
:10131E0000436F6E666967206C6F636B210A00571E
:10132E007220656570726F6D0A00205361766520BC
:10133E00656570726F6D210A00457272204D4143D2
:10134E0021004C6F61643E3E002A00CEF8E8E1EACF
:10135E00E00A00202D202575282575290A003C411C
:10136E0030313D003C4130323D003C4130333D0098
:10137E003C4130343D003C4130353D003C21003C89
:10138E005330323D003C5330333D003C5330353DFD
:0D139E00003C5330383D003C5330363D00DC
:063BE200010B00010900C7
:103C1800C28E438910E4F58B758DB8D2ABD28E2253
:0A3C3400E4FEEEC39F50030E80F87B
:013C3E002263
:03001B0002329E10
:10329E00C0E0C083C082C0D0C28E758B00758DB861
:1032AE0020160675A61E75A6E10509D212E50B605D
:1032BE0002050B050EE50E540F7051E50AD394016D
:1032CE004002150AD21EE50E543F7012D2109066BF
:1032DE008EE0600A04F0E0D394B44002D2169066F9
:1032EE0087E0600204F0906104E0600214F09066E2
:1032FE008FE0D394014003E014F0301502050CE585
:10330E000DD394644004D2168002050DE508D394C3
:10331E000140021508D28ED0D0D082D083D0E032B8
:1008D000C291C290D2B5C21B7D027C007F07123B41
:1008E000C58F25E525646060097D017F60123B604E
:1008F000D21BE4FDFC7F0B123BC58F25E52530E6BE
:10090000097D04E4FF123B84D21B7D017C007F073C
:10091000123BC58F25E5257008FD7FFF123B60D295
:100920001B301B03126000C288C2A8C2AA758900CE
:100930001236E690633FE0B4FA06A3E064CE607B33
:10094000E4F52574372525F582E43463F583E4F076
:100950000525E525B443EC90633F74FAF0A374CE0B
:10096000F0A374CCF0906345740AF0E4A3F0A30400
:10097000F0A3F090633B74FFF0A3F0A3F0E4A3F0C6
:100980009063567403F0E4F525E5252401FFE43374
:10099000FE74372525F582E43463F583E0FD123BD0
:1009A0003C0525E525C3944340DFE4F5A775A61E65
:1009B00075A6E1907FF0F0A3F080FE90634A740387
:1009C000F0A374CCF0E4906349F090668CF0A3F04F
:1009D00012306CC2B51237DEC2161239D9D21BC220
:1009E0001DC21C9065777408F09062B57424F0E421
:1009F000A3F090633FE09062B7F0906340E09062B4
:100A0000B8F0906341E09062B9F0906342E0906288
:100A1000BAF0906343E09062BBF0906344E0906270
:100A2000BCF0750A01E4906578F0C217C218C219CB
:100A3000C21A201B18AF25FE7D03122EAFE4FF1251
:100A400031EE7E0F7F4EE4FBFDFC1229E290668EB4
:100A5000E060037401F0E4906104F0F50C906576B9
:100A6000F0F50D123C1875A70775A61E75A6E1D204
:100A7000AFC213E4F50D906104E070031228BB903F
:100A8000668FE06401701D9080007410F09080A863
:100A900074FFF0A3F0A3F0A3F0E490668FF0D21BF4
:100AA000C21CC21D908008E0F52530E405D2177401
:100AB00010F0E52530E508D2199080087420F0E5A3
:100AC0002530E608D2189080087440F0E50CC394F5
:100AD000034019908002E4F0908001F0908000F0D3
:100AE000E50C94064006E4F50C1239D99080A0E09C
:100AF000700312384F9080B8E07003123764908012
:100B0000D0E0700312397D908000E0701330171030
:100B1000122AE9906332EFF0D394004003120026CA
:100B2000908002E07006908000E06005D215020A15
:100B300073C215E4F50C906104E06003020A7320AF
:100B40001B12906579E0600C7E0F7F50122DC7E478
:100B5000906579F0301912122479906332EFF0D356
:100B600094004005E0FF12001F201803020D03123D
:100B700022F2906332EFF07003020A73906376E022
:100B800054BF247F7003020C55147003020C2D24F3
:100B9000026003020C9C201B077E0F7F57122DC79B
:100BA000906682E06003020D0390634EE070069051
:100BB0006352E06067906683E0FF90634EE0B507A4
:100BC00024906684E0FE90634FE0B5061890668539
:100BD000E0FE906350E0B5060C906686E0FE906300
:100BE00051E06E6037906352E06F6003020D039036
:100BF0006684E0FF906353E06F6003020D0390662C
:100C000085E0FF906354E06F6003020D03906686F9
:100C1000E0FF906355E06F6003020D03C21390651F
:100C2000787401F0120020750A01020D0390668E9F
:100C3000E060037401F090667BE0FF906378E06F02
:100C40006003020D0390667BE004F0E4F50A906512
:100C500076F0020D03301303020D03906345E0703C
:100C600003020A739062B4E06008906356741EF049
:100C700080069063567403F0123C49D213E4F50ADF
:100C8000906576F090668704F0E490667AF0A3F0C1
:100C9000201B707E0F7F65122DC7806790668EE0E7
:100CA00060037401F0301352906376E020E74B90BC
:100CB0006378E0FF90667AE0FE6F600D906682E0F8
:100CC0007007EE146F703C801390667AE004F09029
:100CD0006332E0FFD39404400312332E906000741B
:100CE00082F0A37401F0906378E0906002F07E607F
:100CF0007F007D031234D1020A73201306906683AD
:100D000074FFF0201303020E26E50A706E123C3FBA
:100D1000EF60237E647F76906477E02404FD1234D4
:100D2000D1906682E07009906356E0F50A020A737A
:100D3000E4F50A020A73906687E0D3943C403C9045
:100D40006682E070369062B4E0703090668704F09E
:100D5000123139E4906476F0A37412F090667BE06F
:100D6000906478F0A374FDF090610563A201906433
:100D70007A63A2017F12121E698098123AE88F25C9
:100D8000E525B401159060007483F0E4A3F07E6063
:100D90007F007D021234D1020A73E525D39401400D
:100DA0001C9060007483F0A37401F0E52524FEA379
:100DB000F07E607F007D031234D1020A73E50A647D
:100DC000016003020A73906576E004F0201B077E41
:100DD0000F7F6F122DC7906576E0FFD39401400B13
:100DE000906356E0941E5003E004F0EFC394054076
:100DF0000DC213E4906578F0120020020A737C663D
:100E00007D8390634AE0FAA3E0FB7F021236627EA4
:100E1000647F76906477E02404FD1234D1906356A9
:100E2000E0F50A020A73E50A64016003020A73909E
:100E30006578E0146061147003020F2B14700302D4
:100E40000F3D24036003020A73E4F50C906682E010
:100E5000602D90634EE0FCA3E0FDA3E0FEA3E0FF65
:100E6000906683121C5990634A7403F0A374CCF00B
:100E700030B403020A739065787401F0020A73902B
:100E800080027410F09065767401F0750A12906615
:100E90008374FFF0020A73906683E0605D9064766D
:100EA0007480F09064787401F0E4A3F0A304F0A3DC
:100EB000743FF0A3747BF0E4F525747D2525F5825D
:100EC000E43464F583747DF0747E2525F582E43482
:100ED00064F583E4F0E5252407906477F07C667D73
:100EE0008390634AE0FAA3E0FB7F021236627E64DD
:100EF0007F76E5252409FD1234D1906682E06020DA
:100F0000E4906578F0123C49D213E4F50A906576D6
:100F1000F090668704F0E490667AF0A3F0020A731A
:100F2000E4906578F0750A12020A7390657874038C
:100F3000F0F50AC2B57FFF123C34020A73E49065F3
:0D0F400078F01239D9750A12020A7380FE8A
:010F4D002281
:10002600906377E0B444047F0180027F009063769A
:10003600E0B447047E0180027E00EE5F604A906372
:100046003FE0906378F0906340E0906379F09063CE
:1000560041E090637AF0906342E090637BF09063B6
:1000660043E090637CF0906344E090637DF090639E
:10007600777452F09062AE63A2019080A863A201E9
:100086007F06121E690208C6906332E0C3940850C8
:10009600030208CF90633FE0FF906378E06F600350
:1000A6000208CF906340E0FF906379E06F6003023F
:1000B60008CF906341E0FF90637AE06F6003020827
:1000C600CF906342E0FF90637BE06F60030208CF4E
:1000D600906343E0FF90637CE06F60030208CF907B
:1000E6006344E0FF90637DE06F60030208CF906396
:1000F60077E06444701A9080A8E0B4FF139062AE73
:1001060063A2019080A863A2017F06121E69801077
:100116009062B2E09080ACF09062B3E09080ADF077
:1001260090668EE060037401F090668F7464F090C0
:1001360063777452F0906376E0646D60030202693F
:100146007BFF7A0F797A1217CE7BFF7A0F7994901C
:10015600633FE0F52EA3E0F52FA3E0F530A3E0F52D
:1001660031A3E0F532A3E0F5331217CE752EFF75F5
:100176002F0F7530F17531FF75320F7533FD7BFF2B
:100186007A0F79CA1217CE7BFF7A1079061217CE2C
:100196007BFF7A10796C1217CE7BFF7A10799990D3
:1001A6006345E0F52EA3E0F52FA3E0F530A3E0F5D7
:1001B600311217CE7BFF7A1079C390633BE0F52EA0
:1001C600A3E0F52FA3E0F530A3E0F5311217CE7BBF
:1001D600FF7A1079E6906337E0F52EA3E0F52FA3BA
:1001E600E0F530A3E0F5311217CE7BFF7A117903E3
:1001F6001217CE7BFF7A11792E90634EE0F52EA36F
:10020600E0F52FA3E0F530A3E0F5311217CE7BFF22
:100216007A11795C906352E0F52EA3E0F52FA3E006
:10022600F530A3E0F5311217CE7BFF7A11798A906B
:100236006682E0F52E1217CE7BFF7A1179B59066AD
:100246008EE0F52E1217CE7BFF7A1179E89062B414
:10025600E0F52E1217CE1225EA7BFF7A12791A12D2
:1002660017CE22906376E0644C70737E127F20FB7B
:10027600FDFC1229E290637EE0F526A3E0F527E473
:10028600F529E526906380F0A3E527F07E127F5BD3
:100296007C637D807B021229E2E4F528852782852E
:1002A6002683E0FF74802528F582E43463F583EF26
:1002B600F00527E527700205260528E528B410DC99
:1002C6007E127F5E7C637D807B101229E20529E524
:1002D60029C3941040AC7E127F61122DC722906311
:1002E60076E0646C7060F52A7E127F63FBFDFC127B
:1002F60029E2E4F529E4906380F0A3E52AF07E1272
:100306007F5B7C637D807B021229E2E4F528A82AC4
:10031600E6FF74802528F582E43463F583EFF00563
:100326002A0528E528B410E67E127F5E7C637D8070
:100336007B101229E20529E529C3940840B77E12ED
:100346007F61122DC722906376E0644B7061F528B9
:1003560074682528F582E43463F583E060327468B6
:100366002528F582E43463F583E0F4602374682578
:1003760028F582E43463F583E0FF747E2528F58250
:10038600E43463F583E0B507100528E528B408C012
:100396009061047432F00208C69063767421F030DE
:1003A6001B030208C67E127F9E122DC70208C69046
:1003B6006376E0B4521A201B077E127FA6122DC761
:1003C6009063767472F07E637F767D0812344A22DB
:1003D600906376E064497045201B077E127FB11258
:1003E6002DC790637EE0F526A3E0F527E4F5288582
:1003F6002782852683E0FF74802528F582E434630E
:10040600F583EFF00527E527700205260528E52880
:10041600B480DC7E637F767D8A12344A22906376CE
:10042600E064437046201B077E127FB9122DC790E9
:10043600637EE0F526A3E0F527E4F5288527828587
:100446002683E493FF74802528F582E43463F583DC
:10045600EFF00527E527700205260528E528B48074
:10046600DB7E637F767D8A12344A22906376E0646F
:100476005A7053201B077E127FC2122DC790637ECF
:10048600E0F526A3E0F5277C637D807B80AF27AE71
:1004960026123AB4E4F528852782852683E493FF5D
:1004A60074802528F582E43463F583EFF00527E5AB
:1004B60027700205260528E528B480DB7E637F7653
:1004C6007D8A12344A22906376E064446003020512
:1004D6005D90637EE0FF644470030208C6EFB431AA
:1004E6000CC21B7E127FCE122DC70208C690637EF9
:1004F600E0B4300CD21B7E127FDA122DC70208C67A
:1005060090637EE0B4320CD21C7E127FE7122DC7B8
:100516000208C690637EE0B4330CC21C7E127FF5DF
:10052600122DC70208C690637EE0B4340CD21D7E3D
:10053600137F04122DC70208C690637EE0B4350C03
:10054600C21D7E137F11122DC70208C690637EE07E
:10055600FF12001E0208C6906104E07013201B07FC
:100566007E137F1F122DC79063767421F00208C692
:100576009061047432F0906376E0FFB45104C2AF28
:1005860080FEEF64577045201B077E137F2D122DCA
:10059600C790637FE0906332F0E4F528906332E021
:1005A600FFE528C39F40030208C674802528F5820C
:1005B600E43463F583E0FF90637EE0252824ADF5FF
:1005C60082E43461F583EFF0052880D0906376E00D
:1005D60064536003020680201B077E137F38122DAA
:1005E600C790633FE0FF9061B6E06F703C90634058
:1005F600E0FF9061B7E06F7030906341E0FF90617B
:10060600B8E0B50724906342E0FF9061B9E0B50712
:1006160018906343E0FF9061BAE0B5070C9063441D
:10062600E0FF9061BBE06F60169063767421F03056
:100636001B030208C67E137F47122DC70208C6E4B5
:10064600F528E4F50DAF28FE74AD2528F582E434CF
:1006560061F583E0FD123B3C0528E528C394FE4086
:10066600E1C2AFE4907FF0F0A3F0907FFD74AAF0B2
:10067600A374FFF0A37455F080FE906376E0644F98
:10068600705A90637EE0F526A3E0F527E527452618
:10069600700A201B077E137F50122DC7201B077E72
:1006A600137F57122DC7E4F52874802528F582E4B8
:1006B6003463F583E0852782852683F00527E527C1
:1006C600700205260528E528B480DE90668DE024B4
:1006D60080F090668CE03400F00208C6906376E005
:1006E6006445707490637EE0FEA3E0FF907FF0EEB9
:1006F600F0A3EFF0D39400EE94044038907FF0E03E
:10070600FEA3E0FF90668CE0FCA3E0FD9FEC9E401C
:1007160023E42FFFEE3401FED3ED9FEC9E5015C26D
:10072600AF907FFD74AAF0A374FFF0A37455F0E4B4
:10073600F5A780FE7E137F59122DC77BFF7A1379AA
:1007460061907FF0E0F52EA3E0F52F90668CE0F542
:1007560030A3E0F5311217CE906376E0646560034E
:100766000208CF90637EE0FFA3E0907FF0CFF0A376
:10077600EFF0E4F526F527D3907FF1E09527907FFB
:10078600F0E095264020E4F50D2527FFE526340107
:10079600FE852782852683E0FD123B3C0527E5275B
:1007A6007002052680D17E137F6C123558EF4E609D
:1007B60020120003906345EFF0120003906346EFAA
:1007C600F0120003906347EFF0120003906348EFC6
:1007D600F07E137F72123558EF4E602012000390A0
:1007E600634EEFF012000390634FEFF01200039098
:1007F6006350EFF0120003906351EFF07E137F78A1
:10080600123558EF4E6020120003906352EFF0123B
:100816000003906353EFF0120003906354EFF0125D
:100826000003906355EFF07E137F7E123558EF4E2E
:10083600602012000390633BEFF012000390633CCC
:10084600EFF012000390633DEFF012000390633E59
:10085600EFF07E137F84123558EF4E6020120003AE
:10086600906337EFF0120003906338EFF012000345
:10087600906339EFF012000390633AEFF0E4F52845
:10088600E4F50DE5282401FFE433FE74372528F549
:1008960082E43463F583E0FD123B3C0528E528C37A
:1008A600944340DCC2AFE4907FF0F0A3F0907FFD6C
:1008B60074AAF0A374FFF0A37455F0E4F5A780FEC4
:0908C6007E637F767D0812344A3E
:0108CF002206
:103A7C00AE07EEC39430400BEED394395005EE24D0
:103A8C00D0FF22EEC39461400BEED394665005EE4A
:103A9C0024A9FF22EEC39441400BEED3944650056B
:083AAC00EE24C9FF22AF06223F
:103BFE009062ADE004F070069062ACE004F090626A
:0A3C0E00ACE0FEA3E0FF123BA82289
:10000300123BFE123A7CEFC454F0FEC006123BFED4
:08001300123A7CD0E02FFF221D
:10392000E49069B8F0123BFE9069B9EFF0C39430AF
:103930004018E0FFD3943950119069B8E02405F5A0
:1039400082E43461F583EFF080119069B8E02405DA
:10395000F582E43461F583E4F0800C9069B8E0040A
:10396000F0E0D3940840BE752900752A00752B003D
:0C397000E4F52C7B017A61790512214EF0
:01397C002228
:043558008E2B8F2CFB
:10355C009062ACE4F0A374FFF0123BFEEF606EF4EB
:10356C00606B852C82852B83E493B507EC752D015C
:10357C00E52C252DF582E4352BF583E4936025901D
:10358C0062ADE0252DFF9062ACE03400FE123BA84A
:10359C00E52C252DF582E4352BF583E493B5070452
:1035AC00052D80CCE52C252DF582E4352BF583E417
:1035BC009370A6E52D24FFFFE434FFFE9062ADE08E
:1035CC002FF09062ACE03EF07E007F0122E4FEFF23
:0135DC0022CC
:10306C007E137F8A123558EF4E70037F01227E1338
:10307C007F8D123558EF4E600C123BFEEF24D09032
:10308C006682F08005E4906682F07E137F931235A1
:10309C0058EF4E600C123BFEEF24D090668EF08001
:1030AC0005E490668EF07E137F99123558EF4E60D2
:1030BC000C123BFEEF24D024FF92118002C2117E31
:1030CC00137F9F123558EF4E600C123BFEEF24D04D
:1030DC009062B4F08005E49062B4F090633F63A218
:1030EC000190667C63A2017F06121E6930113B7E43
:1030FC00137FA5123558EF4E603012000390667C9A
:10310C00EFF012000390667DEFF012000390667EE4
:10311C00EFF012000390667FEFF0120003906680D0
:0D312C00EFF0120003906681EFF07F0022AB
:103A3300906577E0C3947C40027F0A906577E0FE4F
:103A430004F074B52EF582E43462F583EFF0BF0A17
:103A530027906577E0FF04F074B52FF582E43462B4
:103A6300F583E4F0906577E0FF1235DD90657774B8
:093A730008F09062B6E004F022B4
:1013AB003E2A2C312CCFE0F0E0ECE5F2F0FB20E014
:1013BB00F1E8EDF5F0EEEDEDEEE3EE20EFEEF0F211
:1013CB00E00A003E4C2C4930312C256C752CD1EAAF
:1013DB00EEF0EEF1F2FC20EEE1ECE5EDE02C353039
:1013EB002C3130302C3330302C3630302C313230F5
:1013FB00302C323430302C343830302C39363030CD
:10140B002C31393230302C33383430302C353736B0
:10141B0030302C3131353230300A003E422C4930DD
:10142B00322C2562752CCFF0EEE2E5F0FFF2FC20BA
:10143B0043545320EFF0E820EFE5F0E5E4E0F7E567
:10144B000A003E532C4931312C25752CC7E0E4E5BD
:10145B00F0E6EAE020F1F2E0F0F2E020EFE5F0E573
:10146B00E4E0F7E82028ECF1290A003E4C2C493047
:10147B00342C25732CD0E5E6E8EC20EFE5F0E5E421
:10148B00E0F7E82C3720E1E8F22C3820E1E8F22CE9
:10149B003920E1E8F20A003720E1E8F2003820E1D8
:1014AB00E8F2003920E1E8F2003E4C2C4931302CB7
:1014BB0025732CCAEEEDF2F0EEEBFC20F7E5F2ED26
:1014CB00EEF1F2E82C302DCDE5F220283120F1F2AF
:1014DB00EEEF2DE1E8F2292C312DD7E5F2EDFBE90A
:1014EB0020284556454E292C322DCDE5F7E5F2ED5A
:1014FB00FBE920284F4444292C332DCDE5F220283D
:10150B003220F1F2EEEF2DE1E8F2E0290A00332D63
:10151B00CDE5F220283220F1F2EEEF2DE1E8F2E0FA
:10152B002900302DCDE5F220283120F1F2EEEF2D00
:10153B00E1E8F229003E4C2C4931302C25732CCAA2
:10154B00EEEDF2F0EEEBFC20F7E5F2EDEEF1F2E86A
:10155B002C302DCDE5F22C312DD7E5F2EDFBE9202A
:10156B00284556454E292C322DCDE5F7E5F2EDFBFE
:10157B00E920284F4444292C332DCDE5F220283285
:10158B0020F1F2EEEF2DE1E8F2E0290A00312DD740
:10159B00E5F2EDFBE920284556454E2900322DCDCD
:1015AB00E5F7E5F2EDFBE920284F444429003E42E4
:1015BB002C4932312C2562752CD3E4E0EBFFF2FC85
:1015CB002022F1E1EEE9EDFBE52220EAE0E4F0FB7D
:1015DB000A003E532C4930372C2562752CC4EEF192
:1015EB00F2E0E2EAE020EFF0E820EFF0E8E5ECE5EE
:1015FB00204E20E1E0E9F220283C313236290A0066
:10160B003E532C4930392C2562752CC4EEF1F2E097
:10161B00E2EAE020EFF0E820EFF0E8E5ECE520E18E
:10162B00E0E9F2E02028302DEDE5F220EAEEEDF2D4
:10163B00F0EEEBFF290A003E422C4932302C25629A
:10164B00752CCAEEEDF2F0EEEBFC20E7E0E4E5F0F2
:10165B00E6EAE820EEF2E2E5F2E02028E2FBF7E82A
:10166B00F1EBE5EDEE20256C7520ECF1290A003E3F
:10167B00422C4932302C2562752CCAEEEDF2F0EE7D
:10168B00EBFC20E7E0E4E5F0E6EAE820EEF2E2E549
:10169B00F2E00A003C4930313D003C4930323D001C
:1016AB003C4930333D003C4931313D003C493034FD
:1016BB003D003C4930353D003C4930363D003C490E
:1016CB0031303D003C4932313D003C4930373D0023
:1016DB003C4930393D003C4932303D000AC1F3F4FE
:1016EB00E5F020E7E0EDFFF221000ACFEEEFFBF291
:1016FB00EAE020EFE5F0E5E4E0F7E820EFF0E820A2
:10170B00EDE5E7E0E2E5F0F9E5EDEDEEEC20EFF0ED
:10171B00E8E5ECE521000A2D3E000A4672616D6595
:10172B00206572726F722120000A3C2D00496E6990
:10173B00745443500A004C697374656E5443500AD9
:10174B0000534F434B5F5443505F45535441424CFE
:10175B0049534845440A000A2D3E20000A3C2D20DF
:01176B00007D
:103BE8005266900000000000000000000000000085
:053BF8000000000000C8
:01001E0022BF
:030023000227575A
:0B275700C0E0C083C082C0D075D01865
:10276200209803022833300140A29A920AE599FD8B
:1027720030071A30D00A30050FD29F30090A80562E
:10278200200505D29F20094E531D7F801EA20A30CC
:10279200D001B3500A300513D29F30090E80372082
:1027A2000509D29F300904802DAD99D291300703DB
:1027B200531D7F74A22553F582E43466F583EDF050
:1027C2000553E5516005B51D02D206E553547FD38A
:1027D20095444002D206E54C603D30083AC208AF4B
:1027E200F9EF7F00FEACE9EC7A002400FFEA3ECF6D
:1027F200C39546F546EF9545F545C3E5469488E50C
:102802004594135012E5469548E54595474006859F
:102812004547854648054CE55025E9F5EB30D70993
:10282200E54F25F904F5FB8006E54F25F9F5FBC2D6
:102832009830997C300277300C07309704D20080B0
:102842006DE555C39552401DC202C290D20DD2967B
:10285200D208AFF9EFFEACE9EC7A002400F546EAC3
:102862003EF5458049AF55055574A22FF582E434F3
:1028720067F583E0F55830071953587F30012C2053
:10288200D008200526635880802130051E635880B9
:102892008019300114E5585258300506A2D0929B97
:1028A2008009A2D0B3929B8002D29B855899C2998B
:0928B200D0D0D082D083D0E032F6
:1025EA007BFF7A1379AB1217CE9068A2E0FEA3E0C4
:1025FA00FFC3E49FFFE49EFEAB07FA3395E0F9F8C8
:10260A007F007E8C7D0A7C00121BA88F318E308D54
:10261A002F8C2E7BFF7A1379CE1217CE7BFF7A147A
:10262A007926A20CE433F52E1217CEAE49AF4A7CB6
:10263A00007D0A121AC88E2E8F2F7BFF7A14794DCD
:10264A001217CE300714752EFF752F147530A27B22
:10265A00FF7A1479761217CE8029200E14752EFF70
:10266A00752F147530A87BFF7A1479761217CE80ED
:10267A0012752EFF752F147530AE7BFF7A1479769A
:10268A001217CE300E14752EFF752F157530197B63
:10269A00FF7A1479B41217CE8040200114752EFFE8
:1026AA00752F1575302D7BFF7A1479B41217CE80E9
:1026BA0029300514752EFF752F157530987BFF7A12
:1026CA001579401217CE8012752EFF752F157530A9
:1026DA00A87BFF7A1579401217CE7BFF7A1579B954
:1026EA00A209E433F52E1217CE7BFF7A1579DD8520
:1026FA00442E1217CE7BFF7A16790B85512E1217AC
:10270A00CED3E54E9400E54D94004031E54E9488D1
:10271A00E54D94135027A20FE433F52EAE4DAF4E7C
:10272A00E4FCFD7B0AFAF9F8121BA88F328E318D70
:10273A00308C2F7BFF7A1679421217CE227BFF7AD2
:0D274A0016797AA20FE433F52E1217CE2275
:101F77007E167F9F123558EF4E600B1239209069FD
:101F8700B4121C59800A9069B4121C6500002580A0
:101F97009069B4E0F8A3E0F9A3E0FAA3E0FB7F00BF
:101FA7007E8C7D0A7C00121BA8121C3A9068A2EE58
:101FB700F0A3EFF0E47B0AFAF9F89069B4E0FCA328
:101FC700E0FDA3E0FEA3E0FF121BA8A804A905AA51
:101FD70006AB07E47FB87E88FDFC121BA88E4F8FE7
:101FE70050740A2550F550E4354FF54F7E167FA5FE
:101FF700123558EF4E600C123BFEEF24D024FF92AF
:102007000C8002C20C7E167FAB123558EF4E601261
:10201700123920E47B64FAF9F8121B1D8E498F4AA6
:102027008005E4F549F54A7E167FB1123558EF4E23
:102037006012123920E47B0AFAF9F8121B1D8E4947
:102047008F4A8005E4F549F54AC20E7E167FB7121E
:102057003558EF4E600A123BFEEF24D0F558800347
:10206700755808E558B40704D207800BE558B4083B
:1020770004C2078002D20E7E167FBD123558EF4E7E
:10208700600C123BFEEF24D024FF92018002C201B4
:102097007E167FC3123558EF4E600C123BFEEF24BD
:1020A700D024FF92058002C205C2017E167FC912A5
:1020B7003558EF4E600A123BFEEF24D0F5588003E7
:1020C700E4F558E558B40106D201D2058009E55870
:1020D700B40204D201C205C2093001157E167FCFB2
:1020E700123558EF4E600A123BFEEF24D024FF92C0
:1020F700097E167FD5123558EF4E60071239208FAB
:102107004480037544407E167FDB123558EF4E60DE
:10211700071239208F518003E4F5517E167FE112B3
:102127003558EF4E600C123BFEEF24D024FF920F80
:102137008002C20F300F08754D13754E888005E475
:06214700F54DF54E7F008E
:01214D00226F
:103B1400C2A9438902758C48758A4875D90475DB36
:103B24004875DC4875DD4875DE48E4F5E9F5F9C209
:083B3400D9C2DAD28CD2DE22E4
:1037DE00C202C20DE4F555F552F553C204C200D231
:1037EE0097D296755609121F77C2ADE4F5C9D2CDA0
:1037FE00D2CCC2C9C2CAF5CDF5CC9068A2E0F5CB49
:10380E00A3E0F5CA85CBCD85CACCE4F598D29EC28D
:10381E009F20070B5387BF200E03300502D29F4314
:10382E008740C29FC2ACC298C29975B81075B710C6
:10383E00D2CAD29CD2AC123B14C2D9C208754C016A
:01384E002257
:01001F0022BE
:10313900E4FF0F2405F582E43461F583E556F00FC9
:1031490074052401F582E43461F583E4F07C667D3D
:1031590095FEED1DAA0470011CF5828A83E0FBAA85
:10316900070F74052AF582E43461F583EBF00EBE8E
:1031790004E07C667D99E4FEED1DAA0470011CF54E
:10318900828A83E0FBAA070F74052AF582E4346179
:10319900F583EBF00EBE04E07C667D9DE4FEED1D3B
:1031A900AA0470011CF5828A83E0FBAA070F740543
:1031B9002AF582E43461F583EBF00EBE04E07C6607
:1031C9007DA1E4FEED1DAA0470011CF5828A83E04D
:1031D900FBAA070F74052AF582E43461F583EBF045
:0431E9000EBE04E032
:0131ED0022BF
:0C3C2800D299D290300F02D204C20622C2
:073C4900D2CAD29CD2AC22CA
:10332E008F26300B030233BD30020E301B030233E7
:10333E00BD7E167FE7122DC72230040B201B707E38
:10334E00167FF5122DC722906379E0F556E52624F7
:10335E00FCFFF5527D7A758363058263A201906747
:10336E00A263A201121E69E4F555D202C296300C78
:10337E0002D200E54A4549601EC2DAE54A25E9F562
:10338E00EC30D709E54925F904F5FC8006E5492519
:10339E00F9F5FCD2038003123C28201B107E177F08
:1033AE00217C677DA2E52624FCFB1229E2C20D22B8
:102CDD00A20672D94003022DC4E553547F940050CF
:102CED0003022D91C291C2AF855357635380535345
:102CFD0080D2AF300B1DE557548024A2F582E43409
:102D0D0066F58363A2019068A863A201AF57121EF6
:102D1D00698065E4906476F0A20482D95005C204FE
:102D2D007420F0E557547FFF906477F090667BE058
:102D3D00906478F0A3E556F0E557548024A2F5820F
:102D4D00E43466F58363A20190647A63A201121ED6
:102D5D0069201B24309F077E177F25122DC77E17F4
:102D6D007F34E557548024A2F582E43466AD82FCAD
:102D7D00E557547FFB1229E2C206C2D9C29FE5571F
:102D8D00547FFF22201B0C309F077E177F25122DAD
:102D9D00C7C29F30D91D30041AC2049064767420C6
:102DAD00F0E4A3F090667BE0906478F0A3E556F034
:0A2DBD007F0122C2D9C2067F002266
:0100200022BD
:1028BB003010489080E8E0700F1238BD301D077E55
:1028CB00177F38122DC7C20B9080E8E0B40E129020
:1028DB0080037408F0301D077E177F41122DC7C28D
:1028EB000B9080E8E0B4060F200B0C301D077E1711
:1028FB007F4C122DC7D20BC210054BE54CC3946411
:10290B00402F201B097D02AF48AE47122EAFE54882
:10291B0025E0F54EE54733F54DC3E54E9464E54DA3
:10292B0094005006754D00754E64E4F547F548F577
:10293B004C300B74200207122F908F268003E4F586
:10294B0026E5266047301D0C7E177F627C687DA8CC
:10295B00FB1229E2E5E92410F5EB30D708E5F92461
:10296B0028F5FB8006E5F92427F5FB9068A863A200
:10297B00019067A263A201AF26121E69852652E45D
:10298B00F555D290C291D202C296D299122CDD8FFC
:10299B0057E5576013122BED301D0D7E177F677CAB
:1029AB00687DA8AB571229E2300008209705C200BA
:1029BB00123C2830030A30DA07C2DAC203123C2871
:1029CB00300210E54BD39414400CC202C290D29645
:0629DB00C29922E4F54B55
:0129E10022D3
:0A3C3F00200B04122CDD227F00226E
:103AE800300B037F0022300D20C20D300F06E54E4B
:103AF80025E9F5EB30D709E54D25F904F5FB8006F6
:0C3B0800E54D25F9F5FB7F01227F00222E
:1039D9009080007480F090633763A201F583F582CB
:1039E90063A2017F08121E6990633F63A201908060
:1039F9008863A2017F0A121E699080927407F0A35E
:103A090074D0F0A37406F0906349E0FF9080B1F0A0
:103A19009080E1EFF09080957455F0A3F0908000CC
:0A3A29007401F090800974F0F0229F
:10384F00908009E04410F09080A0E070609080A11B
:10385F007482F09080A874FFF0A3F0A3F0A3F07F20
:10386F00039080AEEFF0A374CBF09080007402F061
:10387F009069A8121C65000000009069A8E0908074
:10388F0040F09069A9E0908041F09069AAE09080A3
:10389F0042F09069ABE0908043F0A3E4F0A3F0A373
:0D38AF00F0A3F0908018F0A3F0A3F0A3F0B8
:0138BC0022E9
:10397D00908009E04440F09080D17482F07F0390F4
:10398D0080DEEFF0A374CCF09080027402F09069A9
:10399D00AC121C65000000009069ACE0908058F0FE
:1039AD009069ADE0908059F09069AEE090805AF04A
:1039BD009069AFE090805BF0A3E4F0A3F0A3F0A3D7
:0B39CD00F0908030F0A3F0A3F0A3F016
:0139D80022CC
:10376400908009E04420F09080B8E0706C9080B9BB
:103774007482F07F039080C6EFF07FCDA3EFF07FDB
:10378400039080C4EFF0A374CDF09080C074FFF078
:10379400A3F0A3F0A3F09080017402F09069B0123A
:1037A4001C65000000009069B0E090804CF09069C6
:1037B400B1E090804DF09069B2E090804EF0906955
:1037C400B3E090804FF0A3E4F0A3F0A3F0A3F09053
:0937D4008024F0A3F0A3F0A3F09F
:0137DD0022C9
:103662008C268D27A907EAFDE975F018A424ACFF82
:10367200E5F034808F82F583EDF0EBFDE975F0180B
:10368200A4FFAEF024ACFBEE34808B82F583A3ED75
:10369200F08527828C83E0FDEF24A8FFEE3480FEC4
:1036A2008F82F583EDF08527828C83A3E08F828E53
:1036B20083A3F0852782852683A3A3E0FDE975F025
:1036C20018A424A8FFE5F03480FE8F82F583A3A31B
:1036D200EDF08527828C83A3A3A3E08F828E83A340
:0436E200A3A3F0228C
:06344A008D2BAB07AA0662
:10345000908000E030E5079065797401F022906972
:10346000A8E0FCA3E0FDA3E0FEA3E0F52F8E2E8DE7
:103470002D8C2CAE02AF038E838F8263A201E52ECA
:10348000540744C0F583852F8263A201AF2B121E1F
:10349000DBE4FCFDFEE52F252BF52FEE352EF52E7A
:1034A000ED352DF52DEC352CF52C908040E52CF0EC
:1034B000A3E52DF0A3E52EF0A3E52FF09080007496
:1034C00020F0AF2FAE2EAD2DAC2C9069A8121C5958
:0134D00022D9
:0634D1008D26AB07AA06E0
:1034D700908002E030E5079065797403F0229069E7
:1034E700ACE0FCA3E0FDA3E0FEA3E0F52A8E298D66
:1034F700288C27AE02AF038E838F8263A201E52952
:10350700540744D0F583852A8263A201AF26121E91
:10351700DBE4FCFDFEE52A2526F52AEE3529F5290B
:10352700ED3528F528EC3527F527908058E527F065
:10353700A3E528F0A3E529F0A3E52AF0908002741B
:1035470020F0AF2AAE29AD28AC279069AC121C59E0
:013557002251
:0231EE008F262A
:1031F000908001E030E5099065797402F07F00224B
:103200009069B0E0FCA3E0FDA3E0FEA3E0F52A8E08
:10321000298D288C2790667C63A201E529540744F8
:10322000C8F583852A8263A2017F06121EF1E52A72
:103230002406F52AE43529F529E43528F528E4356E
:1032400027F52790657A63A201E529540744C8F55C
:1032500083852A8263A201AF26121EF1E4FCFDFEE3
:10326000E52A2526F52AEE3529F529ED3528F52814
:10327000EC3527F52790804CE527F0A3E528F0A34F
:10328000E529F0A3E52AF09080017420F0AF2AAE82
:0D32900029AD28AC279069B0121C59AF265B
:01329D00220E
:102AE9009081E0E0F526052605260526052605261A
:102AF90005260526052605260526908010E0F529D8
:102B0900A3E0F52AA3E0F52BA3E0F52C9081E1E001
:102B1900F526052605260526052605260526052664
:102B2900052605260526908014E0F52DA3E0F52E4F
:102B3900A3E0F52FA3E0F530E52FB52B08E530B577
:102B49002C037F0022E4F526E52F540744E0F583A2
:102B590085308263A20190637663A2017F08121F08
:102B69002190637863A2019062AE63A2017F06128D
:102B79001E69906376E0F527A3E0F528E4F5269031
:102B89006376E0702AA3E024F8F526E52F5407447C
:102B9900E0F58385308274082582F582E43583F572
:102BA9008363A20190637663A201AF26121F21AE4F
:102BB90027E4FCFDE5302528F530E52F3EF52FED1E
:102BC900352EF52EEC352DF52D908014E52DF0A33D
:102BD900E52EF0A3E52FF0A3E530F09080007440D6
:032BE900F0AF2624
:012BEC0022C6
:1022F2009081E6E0F5260526052605260526052613
:1023020005260526052605260526908028E0F529BE
:10231200A3E0F52AA3E0F52BA3E0F52C9081E7E0FA
:10232200F526052605260526052605260526052663
:1023320005260526052690802CE0F52DA3E0F52E36
:10234200A3E0F52FA3E0F530E4F526E52FB52B0A3F
:10235200E530B52C05C21802245EE52F540744F07F
:10236200F58385308263A20190637663A2017F08C0
:10237200121F21906376E0F527A3E0F528E52845B2
:102382002770099080027410F07F0022906683E02B
:10239200FFF46030906378E06F600302242590665A
:1023A20084E0FF906379E06F7079906685E0FF903A
:1023B200637AE06F706D906686E0FF90637BE06FFA
:1023C2006031805F906378E0906683F0906379E09B
:1023D200906684F090637AE0906685F090637BE08B
:1023E200906686F090637CE0FFA3E090634ACFF0B2
:1023F200A3EFF0906376E0702AA3E024F8F526E5D7
:102402002F540744F0F58385308274082582F582C3
:10241200E43583F58363A20190637663A201AF265C
:10242200121F21AE27E4FCFDE5302528F530E52F0B
:102432003EF52FED352EF52EEC352DF52DAF2CAECC
:102442002BAD2AAC29AB30AA2FA92EA82DD3121C52
:102452004840099080027410F07F002290802CE5A1
:102462002DF0A3E52EF0A3E52FF0A3E530F0908048
:06247200027440F0AF26E9
:012478002241
:102479009081E3E0F526052605260526052605268D
:102489000526052605260526052690801CE0F52942
:10249900A3E0F52AA3E0F52BA3E0F52C9081E4E075
:1024A900F5260526052605260526052605260526DB
:1024B900052605260526908020E0F52DA3E0F52EBA
:1024C900A3E0F52FA3E0F530E4F526E52FB52B0AB7
:1024D900E530B52C05C2190225CFE52F540744E88C
:1024E900F58385308263A20190600463A2017F0EA7
:1024F900121F37906004E0F527A3E0F52890600CDF
:10250900E0FFF4604A90667CE0FEEF6E7079A3E02C
:10251900FF90600DE06F706F90667EE0FF90600E37
:10252900E06F706390667FE0FF90600FE06F705717
:10253900906680E0FF906010E06F704B906681E0DC
:10254900FF906011E06F703FE4906013F080089095
:10255900601374FFF0D2D9906004E0702AA3E024DC
:10256900F2F526E52F540744E8F583853082740E89
:102579002582F582E43583F58363A20190600463C3
:10258900A201AF26121F37AE27E4FCFDE53025284E
:10259900F530E52F3EF52FED352EF52EEC352DF5E1
:1025A9002DAF2CAE2BAD2AAC29AB30AA2FA92EA862
:1025B9002DD3121C485006E5284527700990800143
:1025C9007410F07F0022908020E52DF0A3E52EF015
:1025D900A3E52FF0A3E530F09080017440F0AF2619
:0125E90022CF
:042DC7008E2B8F2C94
:102DCB00908000E030E5079065797401F0229069FE
:102DDB00A8E0FCA3E0FDA3E0FEA3E0F5328E318D6D
:102DEB00308C2FE532FFE5315407FEE42FF52EEE44
:102DFB0034C0F52D852E82F5837423F0052EE52E38
:102E0B007002052D532DC7F582852D83740AF005AD
:102E1B002EE52E7002052D532DC790633F63A20143
:102E2B00852D83852E8263A2017F06121EDB74061D
:102E3B00252EF52EE4352DF52D852B83852C8263E0
:102E4B00A201852D83852E8263A201121EBFE4FC95
:102E5B00FDFE9069A8E0F8A3E0F9A3E0FAA3E02F48
:102E6B00FFEE3AFEED39FDEC38FCEF2408FFE43EB3
:102E7B00FEE43DFDE43CFC9069A8121C599069A846
:102E8B00E0908040F09069A9E0908041F09069AAB1
:102E9B00E0908042F09069ABE0908043F09080002E
:032EAB007420F0A0
:012EAE002201
:0A29E2008E2B8F2C8C2D8D2E8B2F49
:1029EC00908000E030E5079065797401F0229069E1
:1029FC00A8E0FCA3E0FDA3E0FEA3E0F5358E348D4A
:102A0C00338C32E535FFE5345407FEE42FF531EE17
:102A1C0034C0F530853182F5837423F00531E5310E
:102A2C00700205305330C7F582853083740AF00587
:102A3C0031E531700205305330C790633F63A2011A
:102A4C0085308385318263A2017F06121EDB7406FA
:102A5C002531F531E43530F530852B83852C8263B7
:102A6C00A20185308385318263A201121EBF8F368D
:102A7C00EF2531F531E43530F530E52F6017852D34
:102A8C0083852E8263A20185308385318263A20106
:102A9C00AF2F121EDBE5362408252FF52FFFE4FCA3
:102AAC00FDFEE5352FF535EE3534F534ED3533F5E2
:102ABC0033EC3532F532908040E532F0A3E533F05B
:102ACC00A3E534F0A3E535F09080007420F0AF3529
:0C2ADC00AE34AD33AC329069A8121C5926
:012AE80022CB
:0235DD008F3F1E
:1035DF00908000E030E5079065797401F0229069E2
:1035EF00A8E0FCA3E0FDA3E0FEA3E0F5438E428D2F
:1035FF00418C40E543FFE5425407FEE42FFFEE34D4
:10360F00C09062B563A201F5838F8263A201AF3FC1
:10361F00121EDBE4FCFDFEE543253FF543EE35428C
:10362F00F542ED3541F541EC3540F540908040E5F0
:10363F0040F0A3E541F0A3E542F0A3E543F090800D
:10364F00007420F0AF43AE42AD41AC409069A81278
:02365F001C59F4
:013661002246
:062EAF008E278F28AB0501
:102EB500908000E030E5079065797401F022906913
:102EC500A8E0FCA3E0FDA3E0FEA3E0F52E8E2D8D8A
:102ED5002C8C2BE52EFFE52D5407FEE42FF52AEE6D
:102EE50034C0F529852A82F5837423F0052AE52A5D
:102EF500700205295329C7F582852983EBF0052A38
:102F0500E52A7002052990633F63A201852983851F
:102F15002A8263A2017F06121EDB7406252AF52A82
:102F2500E43529F5295329C7E527852A828529838B
:102F3500F0052AE52A700205295329C7F582852956
:102F450083E528F0052AE52A700205295329C7E5F6
:102F55002E240AF52EE4352DF52DE4352CF52CE43B
:102F6500352BF52B908040E52BF0A3E52CF0A3E560
:102F75002DF0A3E52EF09080007420F0AF2EAE2D3D
:0A2F8500AD2CAC2B9069A8121C596A
:012F8F00221F
:1038BD00908009E04480F09080E97441F07F099098
:1038CD0080F6EFF0A37464F09080037402F09080A2
:1038DD0003E020E1F99068A4121C6500000000903F
:1038ED0068A4E0908064F09068A5E0908065F09009
:1038FD0068A6E0908066F09068A7E0908067F0A3DE
:10390D00E4F0A3F0A3F0A3F090803CF0A3F0A3F0BB
:02391D00A3F015
:01391F002285
:102F90009081E9E0F527052705270527052705275F
:102FA00005270527052705270527908034E0F52804
:102FB000A3E0F529A3E0F52AA3E0F52B9081EAE050
:102FC000F5270527052705270527052705270527B1
:102FD000052705270527908038E0F52CA3E0F52D7F
:102FE000A3E0F52EA3E0F52FE52EB52A08E52FB5D1
:102FF0002B037F0022AF2FAE2EAD2DAC2CAB2BAA16
:103000002AA929A828D3121C48400AAF2FAE2BEEBC
:103010009FF527800AAF2FEFF404AE2B2EF527E59E
:103020002E540744E0F583852F8263A2019068A89F
:1030300063A201AF27121F4FE4FCFDFEE52F2527F9
:10304000F52FEE352EF52EED352DF52DEC352CF535
:103050002C908038E52CF0A3E52DF0A3E52EF0A30D
:0B306000E52FF09080037440F0AF27D4
:01306B002242
:022BED008F2730
:102BEF009080E8E0640660037FFF229068A4E0FC19
:102BFF00A3E0FDA3E0FEA3E0F52B8E2A8D298C2800
:102C0F00E4FFFEFDFCAB2BAA2AA929A828C3121C9E
:102C1F004870609081F9E0F5289068A4E0FCA3E08B
:102C2F00FDA3E0FEA3E0FFE4FAF9F8EF2401FFEAC9
:102C3F003EFEE93DFDE83CFC9068A4121C599068EB
:102C4F00A4E0FCA3E0FDA3E0FEA3E0FFE4F8EF2483
:102C5F0001FFEA3EFEE93DFDE83CFC9068A4121C32
:102C6F0059908064E0F528A3E0F529A3E0F52AA3A5
:102C7F00E0F52B9068A863A201E52A540744D8F524
:102C8F0083852B8263A201AF27121F09E4FCFDFE8F
:102C9F00E52B2527F52BEE352AF52AED3529F529D4
:102CAF00EC3528F528908064E528F0A3E529F0A3FA
:102CBF00E52AF0A3E52BF09080037420F0AF2BAE44
:0D2CCF002AAD29AC289068A4121C597F0082
:012CDC0022D5
:103BA800A2AF921FC2AF438E2075D2028F828E833E
:0C3BB800E0FFE4F5D2538EDFA21F92AFB5
:013BC40022DE
:103B3C00E5D220E0FBA2AF921FC2AF43D2028F822C
:103B4C008E83EDF075D25063D250A21F92AFE5D2A6
:033B5C0020E0FB6B
:013B5F002243
:1036E600E4FDED2401FFE433FE123BA874372DF50B
:1036F60082E43463F583EFF00DBD3FE6E4FDED248F
:103706007FFFE433FE123BA8742D2DF582E434616D
:10371600F583EFF0742D2DF582E43461F583E070C6
:103726001B742D2DF582E43461F5837420F0742E1C
:103736002DF582E43461F583E4F080040DBD80BE8E
:10374600E49061ACF0FDEDFF7E00123BA874AD2D58
:0D375600F582E43461F583EFF00DBDFEE96E
:013763002243
:023AB4008B2B5A
:103AB600A2AF921FC2AF85A22C53A2FE8E838F8225
:103AC60005A28C838D827409121F65E52B53A2FE15
:103AD60043A220121F6753A2DF852CA2A21F92AF1A
:013AE600FFE0
:013AE70022BC
:103BC500A2AF921FC2AF8C838D82EF121F6543A2F5
:0C3BD50020121F6753A2DFA21F92AFFF57
:013BE10022C1
:023B60008F26AE
:103B6200A2AF921FC2AFE4F5838D827406121F6565
:103B7200E52643A220121F6753A2DFA21F92AF7F46
:013B82000141
:013B8300221F
:023B84008F268A
:103B8600A2AF921FC2AFE4F5838D82740A121F653D
:103B9600E52643A220121F6753A2DFA21F92AF7F22
:013BA600011D
:013BA70022FB
:101D8E00A907E7FFA805EF93C3966008403B74FCD4
:101D9E002FFF80F00F08EF93C3966008402B74FB63
:101DAE002FFF80E00F08EF93C3966008401B74FA74
:101DBE002FFF80D00F08EF93D3966008400B74F975
:101DCE002FFF80C01F1F1F1F1FEF54FEF80303F7C6
:101DDE00E893FC08E893FD08E893FE08E893FF22D9
:101DEE0009E993C39D6008402974FB29F980F10924
:101DFE00E993C39E6008401A74FA29F980E209E952
:101E0E0093D39F6008400B74F929F980D3191919DF
:101E1E001919E9C313C313FF22740093F8ECC39886
:101E2E004024701F740193F8EDC398401970147418
:0E1E3E000293F8EEC398400E7009740393F8F7
:101E4C00EFC39840037F00227F0122EDF8E6F008F3
:101E5C00A3DFFA22EDF8E0F608A3DFFA22E0A36391
:101E6C00A201F0A363A201DFF475A2002263A20118
:101E7C00F0A363A20122E0A363A201F0A363A20179
:101E8C00E0A363A201F0A363A201E463A201F0A3A7
:101E9C0063A201DFE175A20022E0A363A2016DFE43
:101EAC00936CFDEE058393FC158363A201DFEA7549
:101EBC00A200227F00E493A363A201F00F600CA3A5
:101ECC00E583C2E3F58363A20180EA75A20022E0F8
:101EDC00A363A201F0A3E583C2E3F58363A201DF50
:101EEC00EE75A20022E0A363A201F0A3E583C2E495
:101EFC00D2E3F58363A201DFEC75A20022E0A363B9
:101F0C00A201F0A3E58344F8C2E5F58363A201DFE7
:101F1C00EC75A20022E583C2E3F583E0A363A20182
:101F2C00F0A363A201DFEE75A20022E583C2E4D226
:0A1F3C00E3F583E0A363A201F0A324
:101F460063A201DFEC75A20022E58344F8F583E085
:101F5600A363A201F0A363A201DFEE75A20022F93A
:101F660022C002C004C00612FFF0D006D004D00280
:011F76002248
:1033CA000208D0E493A3F8E493A34003F68001F241
:1033DA0008DFF48029E493A3F85407240CC8C33304
:1033EA00C4540F4420C8834004F456800146F6DFD3
:1033FA00E4800B0102040810204080903BE2E47E46
:10340A00019360BCA3FF543F30E509541FFEE493C7
:10341A00A360010ECF54C025E060A840B8E493A38E
:10342A00FAE493A3F8E493A3C8C582C8CAC583CAB9
:10343A00F0A3C8C582C8CAC583CADFE9DEE780BE71
:013BFD0000C7
:101AC800BC000BBE0029EF8DF084FFADF022E4CC02
:101AD800F875F008EF2FFFEE33FEEC33FCEE9DECCB
:101AE800984005FCEE9DFE0FD5F0E9E4CEFD22ED11
:101AF800F8F5F0EE8420D21CFEADF075F008EF2F5B
:101B0800FFED33FD4007985006D5F0F222C398FD4B
:051B18000FD5F0EA22E8
:101B1D00E88FF0A4CC8BF0A42CFCE98EF0A42CFC67
:101B2D008AF0EDA42CFCEA8EF0A4CDA8F08BF0A4E5
:101B3D002DCC3825F0FDE98FF0A42CCD35F0FCEB44
:101B4D008EF0A4FEA9F0EB8FF0A4CFC5F02ECD3909
:0F1B5D00FEE43CFCEAA42DCE35F0FDE43CFC2276
:101B6C0075F008758200EF2FFFEE33FECD33CDCC30
:101B7C0033CCC58233C5829BED9AEC99E5829840B3
:101B8C000CF582EE9BFEED9AFDEC99FC0FD5F0D690
:101B9C00E4CEFBE4CDFAE4CCF9A88222B800C1B9BA
:101BAC000059BA002DEC8BF084CFCECDFCE5F0CBF8
:101BBC00F97818EF2FFFEE33FEED33FDEC33FCEB31
:101BCC0033FB10D703994004EB99FB0FD8E5E4F9EC
:101BDC00FA227818EF2FFFEE33FEED33FDEC33FCD9
:101BEC00C933C910D7059BE99A4007EC9BFCE99ACD
:101BFC00F90FD8E0E4C9FAE4CCFB2275F010EF2F12
:101C0C00FFEE33FEED33FDCC33CCC833C810D70711
:101C1C009BEC9AE899400AED9BFDEC9AFCE899F84C
:0E1C2C000FD5F0DAE4CDFBE4CCFAE4C8F922DF
:0E1C3A00C3E49FFFE49EFEE49DFDE49CFC22BB
:101C4800EB9FF5F0EA9E42F0E99D42F0E89C45F0F2
:011C58002269
:0C1C5900ECF0A3EDF0A3EEF0A3EFF022FE
:101C6500A8828583F0D083D082121C7C121C7C1242
:101C75001C7C121C7CE473E493A3C583C5F0C58367
:101C8500C8C582C8F0A3C583C5F0C583C8C582C8C9
:011C9500222C
:10176C00E53A242EF8E6053A22782B302602782E1C
:10177C00E475F001121CEE021C96201FEB7F2ED29A
:10178C001F8018EF540F2490D43440D4FF30230B17
:10179C00EF24BFB41A0050032461FFE53B6002152F
:1017AC003B053EE53E7002053D30260D782BE47579
:1017BC00F001121CEEEF021CDC023A337403D22649
:1017CC008003E4C226F53A8B2B8A2C892DE4F53B59
:1017DC00F53DF53EE53B60077F201217A780F575B8
:1017EC003CFFC220C21FC221C222C224C225C22772
:1017FC00121775FF700D3026057F001217B8AF3E1B
:10180C00AE3D22B4255FC2D5C223121775FF24D07A
:10181C00B40A00501A75F00A783B30D50508B6FFAB
:10182C000106C6A426F620D5047002D22280D92443
:10183C00CFB41A00EF5004C2E5D2230219B8D2205B
:10184C0080C6D21F80C0D22180BCD2D580BAD2240F
:10185C0080B47F201217A72021077401B53B0040EC
:10186C00F112176CFF1217A70217E0D227D22580AE
:10187C009512176CFB12176CFA12176CF94A4B7015
:10188C000679897A1A7BFF20212EE53B602A7E009F
:10189C008E82758300121CAF60060EEE653C70F0F4
:1018AC00C2D5EBC0E0EAC0E0E9C0E0EE1219FFD00F
:1018BC00E0F9D0E0FAD0E0FB121C96FF60AAEBC076
:1018CC00E0EAC0E0E9C0E01217A7D0E02401F9D0AB
:1018DC00E03400FAD0E0FBE53C0460DCD53CD98078
:1018EC00877BFF7A1979FBD221809C791080027951
:1018FC0008C225C2278008D2D5790A8004790AC289
:10190C00D5E53C047002F53CE4FAFDFEFF12176CC1
:10191C00FC7B0820201312176CFD7B10301F0A1261
:10192C00176CFE12176CFF7B20EC3382D592D550CE
:10193C0013C3E4301F069FFFE49EFEE42020039DAA
:10194C00FDE49CFCE4CBF8C220EC700CCFCECDCCEB
:10195C00E824F8F870F38017C3EF33FFEE33FEED95
:10196C0033FDEC33FCEB33FB994002FB0FD8E9EB76
:10197C00302005F8D0E0C448B220C0E00AEC4D4E4F
:10198C004F78207B0070C2EAB53C0040BCC0E0122E
:10199C001A01D0F0D0E0202004C4C0E0C4B220C0B2
:1019AC00F0121790D0F0D5F0EB0217E0121D4D1885
:1019BC007D5318F758184E4C184A4218FB4F190310
:0F19CC004419034918634319095518ED4618EDDE
:1019DB004518ED471AA95018522D18562E18792B69
:1019EB00185A231877201A922A18124800001871D7
:1019FB003F3F3F00790AA2D5202214302409B910A9
:101A0B00020404B9080104A2D520250250010420C8
:101A1B0021689221B53B005034C0E07F2030221961
:101A2B007F30A22172257224500F121A58C221C284
:101A3B0025C224C2277F30800F302403E9C0E01277
:101A4B0017A7302403D0E0F9D0E0B53BCC302417F6
:101A5B007F30B9100C1217A77F583023077F78807F
:101A6B0003B908031217A73021057F2D0217A77F93
:101A7B00202027F87F2B2025F322922180CF286E60
:101A8B00756C6C2900D22012176C3020F8C22078AC
:101A9B003B30D50108F60218122D50434958121746
:101AAB006C2403B405004001E4901AA49312179818
:0D1ABB00743A121798D222753B040218F7F6
:10214E008B268A278928E4F532F531F530F52FF5FF
:10215E002DF52EE52A452B45296012EBC0E0EAC08D
:10216E00E0E9C0E0AB29AA2AA92B121CFEAB26057A
:10217E0028E528AA277002052714F9121C96F533B4
:10218E00C394094007E533D3940D40E1E533642051
:10219E0060DBE533B42D05432E038016E533B42BF7
:1021AE0005432E01800C74FF2528F52874FF352772
:1021BE00F527E52C60046410703FAB26AA27A928EA
:1021CE00121C9664306009E52C702E752C0A80293D
:1021DE00900001121CAFFF64786004EFB4581343F3
:1021EE002E01752C1074022528F528E43527F527C5
:1021FE008007E52C7003752C08AB260528E528AA68
:10220E00277002052714F9121C96F533C39461400A
:10221E000AE533D3947A50035333DF74D02533F564
:10222E0033C3940A400CE5339411406D74F9253391
:10223E00F533E533D3952C5060432E018532378527
:10224E003136853035852F34AF2C7E00E4FCFDAB66
:10225E0032AA31A930A82F121B1DC8ECC8C9EDC96E
:10226E00CAEECACBEFCBE4FCFDFEEB2533F532EE26
:10227E003AF531ED39F530EC38F52FAF32AE31ADF0
:10228E0030FCAB37AA36A935A834D3121C485003FC
:10229E00022207432E04022207E52E20E003E480EB
:1022AE002DE52A452B4529601EAB26E52824FFF98E
:1022BE00E52734FFFAEBC0E0EAC0E0E9C0E0AB2965
:1022CE00AA2AA92B121CFEE52E30E20774FFFFFE90
:1022DE00FDFC22E52EAF32AE31AD30AC2F30E10336
:0422EE00021C3A2272
:101C9600BB010689828A83E0225002E722BBFE024C
:091CA600E32289828A83E493227F
:101CAF00BB010CE58229F582E5833AF583E02250EA
:101CBF0006E92582F8E622BBFE06E92582F8E22234
:0D1CCF00E58229F582E5833AF583E493224E
:101CDC00BB010689828A83F0225002F722BBFE01E7
:021CEC00F322E1
:101CEE00FAE6FB0808E6F925F0F618E6CA3AF622F7
:101CFE00BB011A89828A83D0F0D0E0F8D0E0F9D007
:101D0E00E0FAD0E0FBE8C0E0C0F0021D7C5016E91E
:101D1E00F8D083D082D0E0F9D0E0FAD0E0FBC082D8
:101D2E00C083021D73BBFE16E9F8D083D082D0E0CB
:0F1D3E00F9D0E0FAD0E0FBC082C083021D8522FD
:101D4D00D083D082F8E4937012740193700DA3A325
:101D5D0093F8740193F5828883E473740293686039
:061D6D00EFA3A3A380DF39
:091D7300EBF608EAF608E9F62295
:091D7C00EBF0A3EAF0A3E9F02268
:091D8500EBF208EAF208E9F2228F
:00000001FF
